:020000040000FA
:100000008A110A12AD2C0000F20003088301A0003F
:100010000A08A1000408A2000B1900000B18000038
:100020008B180000831203138A110A128C196020A6
:100030000C1B00008C1A00000C1A00000C190000A8
:100040008C1800000C1800000D1800008301220815
:10005000840021088A0020088300F20E720E090035
:1000C000831603171008110583128A110A120319E7
:1000D0008528AB008A110A122B19CF208A110A1227
:1000E0002B1889208A110A12AB19DB208A110A12F7
:1000F000AB1ABB208A110A12AB18C2208A110A124D
:100100002B1AAF208A110A126028831203138C1154
:100110000800AC01C4018316901190119011901148
:100120000830A100B830A2008830A000C030A6007E
:100130000830A40096019001831203138C118316DA
:100140000317063098003B309100FF3093000130D8
:10015000970083120130AD000313031708008316C4
:1001600011121012101111159514831203138C1112
:1001700003174414080083169012831203138C1182
:1001800003170800831690101208130592018312BA
:1001900003138C110317B000831203170800831692
:1001A00011111011101211169510831203138C11D6
:1001B0000317C40108008317831603171408A03E11
:1001C000840083120008A000840A0008A100840AA9
:1001D0000008A2008316031714089011831203135A
:1001E0008C110317C50020083C39B100243A8A114C
:1001F0000A12031928293108043A8A110A1203192C
:1002000008293108343A8A110A1203198A29080088
:1002100045088A110A12031D1D292E08213A8A1148
:100220000A12031D132983160830A1008830A0008C
:100230008A110A12831282290800083A8A110A12C6
:10024000031D232908004508103A03190800080077
:10025000450818398A110A12031D7B292E08063A0F
:100260008A110A12031D38298A110A127E247A295A
:100270002E08663A8A110A12031D44298A110A12AD
:100280007E248A110A127A292E08053A8A110A1246
:10029000031D50298A110A127B238A110A127A2916
:1002A0002E08033A8A110A12031D59298A110A12CB
:1002B0007A292E08013A8A110A12031D7729270884
:1002C000013A8A110A12031D6B298316191483122D
:1002D0008A110A127A292708023A8A110A12031D82
:1002E0007A2983161A1483128A110A127A298A1516
:1002F0000A12BD280800083A8A110A12031D812932
:100300000800080083160317A501C830A400831253
:10031000AE0108008317220884000008A300840AA5
:100320000008A400840A0008A500840A0008A600AA
:10033000840A0008A700840A0008A800840A0008AC
:10034000A900840A0008AA0083160830A100A400AE
:1003500083122308213A88300319C8308316A0007D
:1003600015128312AE0123088A110A120319E82913
:100370002308013A8A110A120319032A2308023AB0
:100380008A110A120319182A2308803A8A110A12BC
:100390000319242A2308813A8A110A120319362ADA
:1003A0002308823A8A110A120319482A230860395D
:1003B000203A8A150A120319002823086039403AA6
:1003C0008A110A12031D0C2B8A110A12AC2C080088
:1003D0002408013A8A110A120319872B2408053AC6
:1003E0008A110A1203196F2B2408093A8A110A127A
:1003F00003191C2C2408033A8A110A120319CB2B67
:100400008A110A120C2B2408013A8A110A120319C4
:10041000C82B24080B3A8A110A1203196B2C2408E2
:10042000033A8A110A1203190C2C8A110A120C2B96
:100430002408013A8A110A120319922B2408033A5C
:100440008A110A120319D62B2408083A8A110A12B3
:1004500003190F2C2408063A8A110A120319522A8A
:100460002408003A8A110A120319112B24080A3AA7
:100470008A110A1203194D2C2408003A8A110A1213
:100480000319202B2408063A8A110A120319522A4A
:100490002408003A8A110A1203194B2B8A110A12F6
:1004A0000C2B08002608223A8A150A120319542830
:1004B0002608213A8A150A120319A22802308A0056
:1004C000031026080339673E03188A0A82000C2BA2
:1004D0006B2A852AB52A0630AE000830B500E63012
:1004E000B2000830B3008A150A12E020B400AA084E
:1004F0008A110A12031D802A29022908031CB4004C
:10050000B40A8A110A127E2408000630AE000310D5
:10051000250D8A150A12CC20B2000310250D013ECC
:10052000CC20B3000230B2070318B30A8A150A12AE
:10053000E020B4000230B202031CB303AA088A11FF
:100540000A120319A62A8A110A12AE2A34082902AD
:100550008A110A120318AE2A2908B4000830B5001F
:10056000B40A8A110A127E2408006630AE002708F9
:100570008A110A12031DC62A2808031DC62A9230B2
:10058000B2000930B3008A110A12FD2A0930B30003
:100590009430B200BB018A150A125621B20A270212
:1005A0008A110A12031DDC2A8A150A125621280212
:1005B0008A110A120319E82AB20ABB0A98303202D9
:1005C0008A110A12031CCB2AAE018A110A120C2BC3
:1005D000063025028A110A12031CF22AAE018A1182
:1005E0000A120C2B250DB3003B088A150A125C2158
:1005F000B200B30A3B085C21B3008A150A125621E7
:10060000B40029022908031CB4000830B500B40A5C
:100610008A110A127E240800831603171814831205
:100620000800831626088400831283172D08800093
:10063000840A800183160230A500C830A400080097
:1006400083161708023A8A110A12031D2D2B8312F2
:1006500027088A110A12031D2D2B83161708033A47
:100660008A110A12031D0C2B83122708003C8A11E1
:100670000A12031C0C2B2708383E8400831700083D
:10068000F000831626088400700880000230A50060
:10069000C830A40008000F302705013A8A110A1259
:1006A0000319602B0F302705023A8A110A12031D25
:1006B0000C2B031083161A1803148A110A12642BC8
:1006C0000310831619180314260884008001800D76
:1006D000840A80010230A500C830A4000800250863
:1006E000AF008A110A12AF1B0C2B8A110A12822149
:1006F0000530AE000800AE01AC012F08831696004D
:100700008A110A120319862B023097000800250867
:10071000013A8A110A12031D0C2BAD108A110A121C
:100720008221080025088A110A12031D0C2B2608B5
:10073000031D0C2B831603301705023A8A110A1287
:10074000031DAD2B83120F302705031DAD2B831620
:1007500018108A110A128221080083160330170527
:10076000033A8A110A12031D0C2B83120F3027053E
:10077000023C8A110A12031C0C2B83170F30270529
:100780008316983E840000108A110A128221080004
:100790008A110A120C2B2508013A8A110A12031D2C
:1007A0000C2BAD148A110A128221080025088A1127
:1007B0000A12031D0C2B2608031D0C2B8316033075
:1007C0001705023A8A110A12031DF12B83120F300A
:1007D0002705031DF12B831618148A110A12822192
:1007E0000800831603301705033A8A110A12031D05
:1007F0000C2B83120F302705023C8A110A12031CAE
:100800000C2B83170F3027058316983E84000014A5
:100810008A110A12822108008A110A120C2B8316EF
:1008200026088400831283172C0880008316013069
:10083000A500C830A40008002508013C8A110A124E
:10084000031C0C2B2508AC008A110A1203192B2C4F
:100850008316033097008A110A1282218316031728
:10086000C830AA000830A9008830A8000830AD00C0
:10087000D030AE004830AC00D830B2000830B10003
:100880008830B0000830B500D830B6004830B40029
:100890000E3099000E309A00080083161708033AAC
:1008A0008A110A12031D0C2B83122708003C8A119F
:1008B0000A12031C0C2B2708383E840083170008FB
:1008C000F000831626088400700880000130A5001F
:1008D000C830A40008008316170883120339033AAE
:1008E0008A110A12031D0C2B2708383E8400831737
:1008F000250880008A110A12822108008316031736
:1009000083172608840083120317B70137083502BE
:100910008A110A120319A02C8A110A12B40B932C03
:100920008A110A129F2C8A150A12E0208000B70A49
:10093000840A8A110A12B20F862CB30A862CAE01E1
:1009400037088316A5004030240640398838A400B3
:0A0950008A110A12080008000800CE
:06095A001E30F200F20B5A
:10096000AF2C8316031381178A150A129E23831650
:1009700003178A110A12640003301705033A031D96
:10098000BB2C831203138501860187018A110A1289
:10099000C9268312031305168A150A1283132330FE
:1009A0008400083064228A110A12031CCC2C8312A2
:1009B000031305128A110A12E82C8A150A128313EE
:1009C00023308400083064228A110A12031C6E2D21
:1009D000831203132308AF002408B1002508B300D5
:1009E0002608B5002708B7002808B900AE01031093
:1009F000A90DAE0DA90DAE0D0130AF07AE0AB001C5
:100A00000310A90DB00DA90DB00D0130B107B00A4A
:100A1000B2010310A90DB20DA90DB20D0130B3073B
:100A2000B20AB4010310A90DB40DA90DB40D013023
:100A3000B507B40AB6010310AA0DB60DAA0DB60D7E
:100A40000130B707B60AB8010310AA0DB80DAA0DF8
:100A5000B80D0130B907B80A8030BA004030BB0089
:100A60002030BC001030BD000830BE000430BF0094
:100A70002E08043C8A110A12031D412DAF080319E8
:100A8000BA013008043C8A110A12031D4A2DB1082C
:100A90000319BB013208043C8A110A12031D532DAD
:100AA000B3080319BC013408043C8A110A12031D5F
:100AB0005C2DB5080319BD013608043C8A110A12E1
:100AC000031D652DB7080319BE013808043C8A11BF
:100AD0000A12031D6E2DB9080319BF01FF30F9007A
:100AE0000430F800831203133A08831203138B13A4
:100AF00086008A110A120D27831203132F08790228
:100B00008A110A120319812E00008A110A12F90BA8
:100B10007E2D8A110A12F80B7E2D8B17FF30F900FB
:100B20000430F800831203133B08831203138B1362
:100B300086008A110A120D278312031331087902E5
:100B40008A110A1203198D2E00008A110A12F90B5C
:100B50009E2D8A110A12F80B9E2D8B17FF30F9007B
:100B60000430F800831203133C08831203138B1321
:100B700086008A110A120D278312031333087902A3
:100B80008A110A120319992E00008A110A12F90B10
:100B9000BE2D8A110A12F80BBE2D8B17FF30F900FB
:100BA0000430F800831203133D08831203138B13E0
:100BB00086008A110A120D27831203133508790261
:100BC0008A110A120319A52E00008A110A12F90BC4
:100BD000DE2D8A110A12F80BDE2D8B17FF30F9007B
:100BE0000430F800831203133E08831203138B139F
:100BF00086008A110A120D2783120313370879021F
:100C00008A110A120319B12E00008A110A12F90B77
:100C1000FE2D8A110A12F80BFE2D8B17FF30F900FA
:100C20000430F800831203133F08831203138B135D
:100C300086008A110A120D278312031339087902DC
:100C40008A110A120319BD2E00008A110A12F90B2B
:100C50001E2E8A110A12F80B1E2E8B1783120313F5
:100C600081018312031381309F0025271F158A11EC
:100C70000A121F19372E1E08A300252783120313FB
:100C800081018312031389309F0025271F158A11C4
:100C90000A121F19472E1E08A400252783120313CA
:100CA00081018312031391309F0025271F158A119C
:100CB0000A121F19572E1E08A50025278312031399
:100CC00081018312031399309F0025271F158A1174
:100CD0000A121F19672E1E08A60025278A150A1258
:100CE000831383120313233084000830E8228A110F
:100CF0000A12031C6E2E8A110A1216278A110A1272
:100D0000DD2C2E0878028A110A12031D852D83120C
:100D10000313860183120313852D300878028A118C
:100D20000A12031DA52D83120313860183120313D8
:100D3000A52D320878028A110A12031DC52D8312CF
:100D40000313860183120313C52D340878028A1118
:100D50000A12031DE52D8312031386018312031368
:100D6000E52D360878028A110A12031D052E83121A
:100D70000313860183120313052E380878028A11A3
:100D80000A12031D252E83120313860183120313F7
:100D9000252E83160313EF308500003086000030C7
:100DA00087008316031302309F00831203139F17DB
:100DB0001F13831603130C1383120313F801F90195
:100DC000AE01AF01B001B101B201B301B401B5018F
:100DD000B601B701B801B9018030BA004030BB009C
:100DE0002030BC001030BD000830BE000430BF0011
:100DF00083120313A301A401A501A601A701A80161
:100E0000A901AA010800FF3083120313F4000000B7
:100E10008A110A12F40B072F080083120313FF3004
:100E2000F4008A110A12F40B112F08000430F400A8
:100E3000FF30F500000000008A110A12F50B1A2F8E
:100E40008A110A12F40B182F08000230F400FF3048
:100E5000F500000000008A110A12F50B292F8A11F3
:080E60000A12F40B272F080011
:101000008A150A122308213A031927288A150A1279
:101010002308223A0319C4288A150A122308233AFE
:101020000319C4288A150A122308A13A0319C428EF
:101030008A150A122308A23A0319C4288A150A122B
:101040002308A33A0319C4288A110A120C2B240876
:10105000013A8A150A120319C4282408023A8A158B
:101060000A120319C4282408033A8A150A1203191C
:10107000C4282408063A8A150A1203195428240899
:10108000093A8A150A120319C72824080A3A8A1548
:101090000A120319C42824080B3A8A150A120319E4
:1010A000C4288A110A120C2B831203170630AE00D3
:1010B0000830B5002608013A8A150A120319732868
:1010C0000310270D8A150A12D620B2000310270D2F
:1010D000013ED620B3008A150A12E020B400B20AFD
:1010E0008A150A1293282608023A8A150A12031949
:1010F0008C280310270D8A150A12D620B20003107F
:10110000270D013ED620B3008A150A12E020B40054
:10111000B20A8A150A1293282608033A8A110A127B
:1011200003190C2B08002A088A150A12031D9D2892
:101130002908340229080318B400B40A8A110A12D3
:101140007E2408000630AE000830B5000A30B20038
:101150000930B3008A150A12E020B400AA088A15E3
:101160000A12031DB72829022908031CB400B40A77
:101170008A110A127E24080008008A110A122E0819
:10118000063A03197E2408008A110A120C2B21301A
:10119000AE00831603170800F00008308A00D43030
:1011A000700703188A0A8200F8340834F000083007
:1011B0008A00DE30700703188A0A8200213409345D
:1011C0008312031733088A00320882001234013474
:1011D0000034013400340034003408340034003466
:1011E0000334003400340034023401340034013458
:1011F0000934023429340034013401340434803495
:1012000032340934043400340034023403340034FA
:101210000034003409342134003401340034013402
:101220002234343400340734053481340334083430
:1012300000340A34073405340134033408340034EC
:101240000A3434340634A034FF3409340134A13470
:10125000013409340234A13400340634A134FF349B
:1012600009340334093404341534803425347F348C
:10127000353400344534FF3475340834953408343B
:101280008134023409340534093406341534803489
:1012900025347F34353400344534FF347534083414
:1012A0009534083491340234C034C03483120317A7
:1012B00033088A0032088200F0000310F00D8A150E
:1012C0000A126F21B600F00A8A150A126F21F00087
:1012D00070088A003608330703188A0A820009302A
:1012E0008A007630700703188A0A82007A3409343B
:1012F000863409349234093498340934BA340934C0
:10130000D6340934E2340934EC34093492340934E3
:10131000FC34093410340A343E340A344A340A3472
:1013200054340A340634033409340434043408349D
:1013300022340334493400344F340034433400340D
:101340006134003472340034643400342D34003499
:1013500055340034533400344234003453340034B0
:101360006534003472340034763400346F34003421
:10137000733400341C3403344D340034613400348D
:101380006E34003475340034653400346C34003409
:101390002034003456340034653400346C34003466
:1013A000653400347A340034203400340C3403348F
:1013B00056340034313400342E34003430340034A8
:1013C000303400340A340334433400346634003497
:1013D0006734003431340034103403344E34003474
:1013E0006F340034743400346834003469340034A9
:1013F0006E34003467340034143403344D34003414
:101400006934003463340034723400346F3400348F
:101410006334003468340034693400347034003488
:101420002E340334503400346934003463340034CF
:10143000313400343634003443340034373400342B
:10144000363400343534003420340034553400341C
:1014500053340034423400342034003449340034EE
:101460004F34003443340034613400347234003477
:101470006434003473340034203400340C340334C6
:1014800056340034313400342E34003430340034D7
:10149000303400340A3403344334003466340034C6
:1014A0006734003431340034103403344E340034A3
:1014B0006F340034743400346834003469340034D8
:0814C0006E340034673400347F
:0814C800030883120317C3009F
:1014D0000408BD00831603178A150A12A81BA02A48
:1014E000290883120317C100C2008A150A120319C2
:1014F000902A831603172A0883120317BE00831746
:101500003E0884000008F1003D088400C31F8313D7
:1015100071088000BD0ABE0A8A150A12C10B7F2A13
:10152000831628084039403A8838A8000830A900B6
:1015300083124208F1004308830071080314080075
:101540008312031743088300031008000308831263
:101550000317C3000408BD00831603178A150A1277
:10156000B01BE22A310883120317C100C2008A159A
:101570000A120319D22A831603173208831203179B
:10158000BE0083173E0884000008F1003D08840077
:10159000C31F831371088000BD0ABE0A8A150A1290
:1015A000C10BC12A831630084039403A8838B00050
:1015B0000830B10083124208F1004308830071082B
:1015C0000314080083120317430883000310080064
:1015D000F100030883120317C30071080F39C1001B
:1015E0000408BE004108831603178A150A12AC1BB3
:1015F0001F2BAD008A150A120319132B2E08831214
:10160000BD008317C31F83133E0884000008F10048
:1016100083173D08840071088000BD0ABE0A8A1540
:101620000A12C10B012B83162C084039403A883826
:10163000AC0083120317430883000314080003104F
:101640000800F100030883120317C30071080F3963
:10165000C1000408BE004108831603178A150A1248
:10166000B41B582BB5008A150A1203194C2B3608E7
:101670008312BD008317C31F83133E088400000834
:10168000F10083173D08840071088000BD0ABE0A7E
:101690008A150A12C10B3A2B831634084039403A96
:1016A0008838B4008312031743088300031408002A
:1016B0000310080083170339983E840000140800C3
:1016C00083170339983E8400001008008312031723
:1016D000441C0800831610111115951463000000B6
:1016E0009510101211161011111108008312031712
:1016F000AD1C08008316951011161012111110114F
:1017000015158312BB018030BC008A150A12BB0B71
:10171000872BBC0B872B8316151108008316031724
:1017200095118312BC01BB018A150A12BB0F962BBF
:10173000BC0F962B8A150A129E23080083160317E6
:101740009701013091009001083095008312AC019F
:101750000130AD00B801B901BA01FF30AE0083120B
:1017600003138C1183168C150B178B170800831627
:0E177000031795119514970103138C110800AF
:044000000034003454
:02400E00FA3F77
:00000001FF
